:1000000087C0A2C0B0C09FC0BDC09DC0D3C0D3C078
:100010009AC0B5C298C097C096C095C094C093C00E
:1000200092C091C090C08FC08EC08DC08CC054C291
:100030008AC089C071060071060071060971060B3D
:1000400071060DA40500930B00700A00CF0A01CFC2
:100050000A00CC0800A10701A10700500900B30C59
:100060000057070001000002000004000008000023
:10007000100000020100010200000400000900005D
:10008000110000240000480000880000080100E87A
:100090000100C80300880700080F00081E00083C84
:1000A000DD0C3A0DA40DEB0D3A0DA10E4E0EA10E76
:1000B00001000200040008000F001E003C00780050
:1000C000F000E00184030807100E201C4038807007
:1000D00000010203040506070203040506070809D8
:1000E00001020304010203040102030401020304E8
:1000F0000405060708090A0B0C0D0E0F101110203D
:1001000040000100010001081020304080FF000184
:1001100011241FBECFEFD4E0DEBFCDBF11E0A0E0C1
:10012000B1E0EAE4FDE102C005900D92A030B10714
:10013000D9F711E0A0E0B1E001C01D92AA30B107EB
:10014000E1F757D300CE5CCF1F920F920FB60F92FC
:1001500011248F9381E0809304018F910F900FBE43
:100160000F901F9018951F920F920FB60F921124A7
:100170008F9382E0809304018F910F900FBE0F90B8
:100180001F9018951F920F920FB60F9211242F9364
:100190003F938F9388E028E130E00FB6F894A8955C
:1001A000209360000FBE8093600083B7817F8460DE
:1001B00083BFFFCF18951F920F920FB60F92112495
:1001C0008F931092B4008091B60082FDFCCF8F9186
:1001D0000F900FBE0F901F901895809164008E7F36
:1001E00080936400F999FECF8BE090E092BD81BDD1
:1001F000F89A80B5813029F482E080BF559A5F9AE1
:1002000005C083E080BF459A579A5D9A613011F42A
:10021000529A5A9A80917F00816080937F008091EA
:100220007A008F7780937A0080917B00806480933E
:100230007B0085E080937C00089580B7877F80BF36
:1002400080B7806880BF08953FB7F894A895982F2D
:100250009770292F206483FF02C0292F2066809188
:100260006000886180936000209360003FBF83B787
:10027000817F866083BF90E008C083B7816083BFC1
:10028000889583B78E7F83BF9F5F9617B0F388E111
:100290000FB6F89480936000109260000FBE08952E
:1002A00064E083E0D1DF80B7806180BF80B7886081
:1002B00080BF08958823B9F45B9A0000109204016E
:1002C000E99A83B7817F866006C083B7816083BF68
:1002D000889583B78E7F83BF809104018823A9F31B
:1002E000E9985B9808958BB18C608BB900001092EF
:1002F00004018DB383608DBB83B7817F866006C0A8
:1003000083B7816083BF889583B78E7F83BF8091D9
:1003100004018823A9F38DB38C7F8DBB8BB1837FC0
:100320008BB9089561E083E08FDF5B9A000089B1AB
:100330005B9883FFF7CF08955B9A0000000089B1B6
:100340005B988095887008955A9A000089B15A98F0
:10035000809584700895CF92DF92EF92FF920F9371
:100360001F93F82EC62ED42EE22E0091610085E058
:1003700090E020E80FB6F89420936100809361002C
:100380000FBE10E015C05C9A80E002C000008F5FD5
:100390008F15E0F35C9880E002C000008F5F8F153E
:1003A000E0F39F5F9C1578F36D2D80E04DDF1F5FBC
:1003B0001E1510F490E0F6CF0F7080E80FB6F89499
:1003C00080936100009361000FBE1F910F91FF9019
:1003D000EF90DF90CF9008956F927F928F929F92CF
:1003E000AF92BF92CF92DF92EF92FF920F931F9343
:1003F000CF93DF93A82E7B013A014901FB011082C4
:1004000088E0B82EDD24C0E0D0E000E0CC2461E03C
:1004100082E01ADF5B9A0000000019B15B9810952A
:100420001870BB2079F0112379F4F70180818F5F78
:100430008083F301D183C083F401C082DD24C0E056
:10044000D0E008C0112331F0FFEFCF3FDF07B1F05C
:10045000219614C0D39480E0082F0F5F883049F4B0
:10046000CA1438F4C39421E040E06CE08AE073DF02
:1004700000E0B12E8AE08D1550F602C0802FECCF3F
:10048000DF91CF911F910F91FF90EF90DF90CF9070
:10049000BF90AF909F908F907F906F9008950F9333
:1004A0001F93182F00E017FF04C021E044E168EC1F
:1004B00005C016FF05C021E044E16EE189E14BDF94
:1004C0000F5F043019F0110F110FEDCF61E086E0DE
:1004D000BBDE1F910F9108951F920F920FB60F92DE
:1004E00011242F933F934F935F936F937F938F9339
:1004F0009F93AF93BF93EF93FF9380910501873054
:1005000061F42D9A419A21E040E062ED8AE023DF18
:100510001092060180B7877F80BF809105018530EA
:10052000A1F480910601893048F02D9A419A21E08A
:1005300040E062ED8AE00FDF2D984198809106013E
:10054000882319F480E180930601809105018630AB
:1005500011F41092060180B7806180BFFF91EF9186
:10056000BF91AF919F918F917F916F915F914F91CB
:100570003F912F910F900FBE0F901F9018951F92D3
:100580000F920FB60F9211242F933F934F935F93C7
:100590006F937F938F939F93AF93BF93EF93FF934B
:1005A000809105018730C1F4809106018F3F29F0C9
:1005B000809106018F5F80930601809101018F5F1A
:1005C0008093010190E08F709070892B29F421E0D5
:1005D00040E061E081E0BFDE809105018530C1F43B
:1005E00080910601882329F0809106018150809333
:1005F0000601809101018F5F8093010190E08F706F
:100600009070892B29F421E040E061E081E0A3DED5
:1006100080910501833009F047C0809108019091D5
:1006200009010197909309018093080180910801C5
:1006300090910901892B61F480910201909103014D
:100640009093090180930801809107018093010133
:10065000209101012223E1F080910601813061F4B3
:1006600085B190E2892785B988B192E0892788B958
:100670002150209301010CC0419A2A3008F42D9A90
:10068000822F815080930101882311F42D98419885
:10069000809100018F5F8093000180FD05C021E003
:1006A00040E061E081E057DE80910501843009F08F
:1006B00042C080910801909109010197909309012E
:1006C000809308018091080190910901892B69F4B8
:1006D0008091020190910301909309018093080198
:1006E000809101018F5F80930101809101018E3023
:1006F00010F01092010180910101813011F42D9AC6
:100700000BC0823011F4419807C0883011F4419A2F
:1007100003C0893009F42D98809100018F5F809388
:10072000000190E08F709070892B29F421E040E067
:1007300061E081E010DE80910501863039F580911D
:10074000080190910901892B49F08091080190914D
:100750000901019790930901809308018091060196
:100760008F3F29F0809106018F5F80930601809171
:1007700000018F5F8093000190E083709070892B5F
:1007800029F421E040E061E081E0E5DD80910501B0
:100790008830F1F4809108019091090101979093BC
:1007A0000901809308018091080190910901892B2A
:1007B00019F483E080930401809100018F5F80939E
:1007C000000180FD05C021E040E061E081E0C3DD83
:1007D000FF91EF91BF91AF919F918F917F916F9119
:1007E0005F914F913F912F910F900FBE0F901F90EF
:1007F0001895A89584B7877F84BF88E10FB6F894D1
:1008000080936000109260000FBE83E090E020E8CB
:100810000FB6F89420936100809361000FBE549A44
:10082000389A259A399A8091640081608093640097
:10083000809164008062809364008091640088608D
:100840008093640080916400846080936400809150
:10085000640080688093640080916400826080936B
:1008600064008091680086608093680080916C00CD
:10087000886180936C0080916D00836080936D002F
:100880007894489B02C028E001C020E0499922608A
:10089000339921603499246030E0C901880F991F91
:1008A000820F931F9C012C5C3F4FF901459154919D
:1008B0009C012A5C3F4FF90185919491FA010995B9
:1008C00061E086E0C1DC21E040E060E184EB43DDF3
:1008D00028E088E190E00FB6F894A8958093600036
:1008E0000FBE2093600083B7817F846083BFFFCFFA
:1008F00021E045E06CE384E02EDD21E040E069E1A9
:100900008CE029DD0895BF92CF92DF92EF92FF92A3
:100910000F931F93CF93DF93182FF92E062FE72EF7
:10092000B42E822FBCDDF999FECFC12FDF2DD2BDB1
:10093000C1BDF89AC0B4802F9E2DFC017F0100E05C
:10094000DD243FC0F7018491C81621F422E044E081
:100950006EE103C021E040E06DE285E0FCDC10E0E8
:100960005B9A0000000089B15B9883FD20C0F7010D
:100970008491F999FECF1FBAD2BDC1BD80BD0FB61B
:10098000F894FA9AF99A0FBECDDC21E04AE064E1CE
:1009900088E2E1DC21E04AE068E284E1DCDC21E09D
:1009A0004AE060E58AE0D7DCDD24D39406C061E04C
:1009B00082E04ADC1F5F123199F60F5F0894E11C58
:1009C000F11C0B1518F4DD2009F4BCCF64E084E0C1
:1009D0003BDC8EDFDF91CF911F910F91FF90EF9065
:1009E000DF90CF90BF900895AC018091B0008260FD
:1009F0008093B00083E08093B3001092B20083B57F
:100A0000826083BD8091700082608093700020E0DE
:100A100030E02DC01092B4008091B60082FDFCCF72
:100A200083B7817F866083BF83B7816083BF8895EA
:100A300083B78E7F83BF5B9A0000000089B15B980B
:100A400083FD13C02D9854DF6DDC88E028E130E091
:100A50000FB6F894A895209360000FBE80936000B5
:100A600083B7817F846083BFFFCF2F5F3F4F241701
:100A7000350780F2809170008D7F8093700008951B
:100A80000F931F93CF93DF93082F162F613011F030
:100A90006330C8F021E040E061E081E05CDCF9997E
:100AA000FECF86E090E092BD81BDF89A80B581309E
:100AB00009F4419A2D9A80E290E096DF41982D98B2
:100AC00080E490E091DF21E040E061E081E043DC00
:100AD000F999FECF86E090E092BD81BDF89A80B58D
:100AE000813009F4419A2D9A802F90E0FC01EE0F9D
:100AF000FF1FE80FF91FEC59FF4F20E034914AEF38
:100B000050E004C0FA013197F1F72F5F2317D0F3BB
:100B1000FC01EE0FFF1FE80FF91FEB59FF4FC591C6
:100B2000D491CE0161DF41982D9821E040E061E051
:100B300085E011DC123018F0CE01489655DFDF91C8
:100B4000CF911F910F9108950F931F93DF93CF9330
:100B500000D000D0CDB7DEB721E040E06AE084E00D
:100B6000FADB80E0A7DB9E012E5F3F4FAE014D5FB9
:100B70005F4FBE016F5F7F4F80E02EDC8981813047
:100B8000B1F400E017E017FF04C021E048E268EC90
:100B900003C021E048E26EE189E1DDDB0F5F083050
:100BA00011F0110FF0CF61E086E04EDB7FC08230A4
:100BB00039F429E94EE060EF70E089E090E062C02E
:100BC000833039F42CE544E06CEE70E088E090E08E
:100BD00059C0843039F424E544E068EE70E087E0E1
:100BE00090E050C0853039F427E544E064EE70E0D1
:100BF00083E090E047C0863039F420ED44E060EEB9
:100C000070E082E090E03EC0873039F429E647E0AA
:100C100067E071E085E090E035C0883039F429E57F
:100C200042E065E071E084E090E02CC0893039F466
:100C300029E942E06EE071E086E090E023C08A306E
:100C400039F425E648E068ED70E081E090E01AC0F4
:100C50008B3039F425E948E060ED70E080E090E009
:100C600011C08C3039F420E442E061E071E08BE0A7
:100C700090E008C08D3041F424E943E06EEF70E06D
:100C80008AE090E040DE12C08E3039F420EA42E083
:100C900063E071E08CE090E0F5CF2ADE61E083E074
:100CA000D3DA26DE61E083E0CFDA22DE88E028E1D5
:100CB00030E00FB6F894A895209360000FBE8093A3
:100CC000600083B7817F846083BFFFCF21E045E070
:100CD00069E18CE040DB21E040E06CE384E03BDB59
:100CE0000895AF92BF92CF92DF92EF92FF920F934F
:100CF0001F93DF93CF9300D000D0CDB7DEB7182F6E
:100D000081E0D8DA8091B60080628093B60080914D
:100D1000B10086608093B1001092B4008091B6005B
:100D200082FDFCCF9E012E5F3F4FAE014D5F5F4FB6
:100D3000BE016F5F7F4F83E04FDB419AC7DF419871
:100D40001123C9F4F999FECF88E090E092BD81BDEE
:100D5000F89AE0B4F999FECF87E090E092BD81BDAA
:100D6000F89A20B5F999FECF89E090E092BD81BD57
:100D7000F89A10B510C0F999FECF83E090E092BDCB
:100D800081BDF89AE0B4F999FECF82E090E092BD7F
:100D900081BDF89A20B549814250420F43704F5FA0
:100DA000212F30E04E9DC00111242817390714F47B
:100DB000FF2405C04E9D802D1124F12EF81AF999BB
:100DC000FECF21E030E032BD21BDF89A80B5F816A3
:100DD00030F4F999FECF32BD21BDF89AF0B44E9DA2
:100DE000002D1124010F043108F003E180E490E0AC
:100DF000FBDDF999FECFF4E0CF2EF0E0DF2ED2BC80
:100E0000C1BCF89A80B58823D9F41F2DE5E0AE2E39
:100E1000E0E0BE2E13C06A81812F32DE101768F425
:100E2000F999FECFB2BCA1BCF89A80B590E0DCDDA8
:100E30001C3018F080E390E0D7DD1E0D011758F745
:100E4000F999FECFD2BCC1BCF89A80B58130D9F4F3
:100E5000102F75E0C72E70E0D72E13C06A81812F46
:100E60000FDEF11668F4F999FECFD2BCC1BCF89A36
:100E700080B590E0B9DD1C3018F080E390E0B4DD7F
:100E80001E191F1558F764E084E0DED931DD88E0D3
:100E900028E130E00FB6F894A895209360000FBECB
:100EA0008093600083B7817F846083BFFFCF0F93FF
:100EB0001F9380E0FFD900E010E05B9A0000000083
:100EC00089B15B9883FD08C0419A2D9A0F5F01316B
:100ED00009F4FCDE10E018C00131D0F42D984198DF
:100EE0001F5F163080F088E028E130E00FB6F894FC
:100EF000A895209360000FBE8093600083B7817F28
:100F0000846083BFFFCF00E061E082E09DD9D5CF50
:100F100061E083E099D980E0CDD92D984198E8DC53
:100F200001DA88E028E130E00FB6F894A895209324
:100F300060000FBE8093600083B7817F846083BFB1
:100F4000FFCFFF920F931F93DF93CF9300D000D07A
:100F50000F92CDB7DEB7F82E83E08093050180E0D5
:100F6000A9D99E012D5F3F4FAE014C5F5F4FBE017F
:100F70006E5F7F4F81E030DA8A81813110F080E14D
:100F80008A838A81813009F07BC08C819D81099799
:100F900008F476C023E045E06EE184E0DCD980E02F
:100FA00089D9C0D993DE419A2D9A00E010E020C083
:100FB00061E082E049D95B9A0000000089B15B984A
:100FC00083FD14C02D98419893DCACD988E028E1CA
:100FD00030E00FB6F894A895209360000FBE809380
:100FE000600083B7817F846083BFFFCF0F5F1F4F97
:100FF0008C819D819695879508171907C8F22D98C1
:10100000419800E010E020C061E082E01DD95B9AC9
:101010000000000089B15B9883FD14C02D984198B1
:1010200067DC80D988E028E130E00FB6F894A89515
:10103000209360000FBE8093600083B7817F84603F
:1010400083BFFFCF0F5F1F4F8C819D819C01369521
:101050002795821B930B0817190708F0A4CFD4CF4C
:1010600021E040E06EE184E076D900FF03C061E05A
:1010700084E002C061E085E0E7D80F5F1F4F02C047
:1010800001E010E08A8190E08017910748F780E046
:1010900011D99E012D5F3F4FAE014C5F5F4FBE01E6
:1010A0006F5F7F4F80E098D98091B6008062809317
:1010B000B6008091B10084608093B1001092B200BC
:1010C0001092B4008091B60082FDFCCFFFDD82E07B
:1010D000809307012A8181E0F816C9F4F092060195
:1010E00081E090E0821B9109880F991FEE27FF276E
:1010F000E81BF90BE055FF4F85919491880F991FDC
:1011000090930901809308012D9A419A10C02430D0
:1011100040F08DE080930701253018F081E1809345
:10112000070182E090E090930901809308012A81F1
:1011300081E090E0821B9109880F991FEE27FF271D
:10114000E81BF90BE055FF4F85919491880F991F8B
:1011500090930301809302018091700081608093DD
:10116000700080E0A7D8809170008E7F809370001F
:101170002D984198BDDBD6D828E088E190E00FB6E5
:10118000F894A895809360000FBE2093600083B709
:10119000817F846083BFFFCF1F93DF93CF9300D005
:1011A00000D0CDB7DEB784E08093050180E082D81F
:1011B0009E012E5F3F4FAE014D5F5F4FBE016F5FDF
:1011C0007F4F83E009D98981813110F080E18983E3
:1011D00011E00EC021E040E06EE184E0BCD810FFD9
:1011E00003C061E084E002C061E085E02DD81F5FAC
:1011F0008981811778F780E05DD894D88091B60016
:1012000080628093B6008091B10082608093B100CB
:101210001092B2001092B4008091B60082FDFCCF13
:1012200055DD81E090E09093090180930801898168
:1012300081508983E82FF0E0EE0FFF1FE055FF4F4C
:101240008591949190930301809302018091020112
:1012500090910301880F991F9093030180930201DD
:101260008091700081608093700080E023D880912D
:1012700070008E7F809370002D98419839DB52D892
:1012800028E088E190E00FB6F894A895809360007C
:101290000FBE2093600083B7817F846083BFFFCF40
:1012A0001F93DF93CF9300D000D00F92CDB7DEB75E
:1012B00088E08093050180E0FDD79E012D5F3F4FC0
:1012C000AE014C5F5F4FBE016F5F7F4F80E084D8FF
:1012D0008981813110F080E189838091B60080623C
:1012E0008093B6008091B10084608093B100109229
:1012F000B2001092B4008091B60082FDFCCF11E0E4
:101300000EC021E040E06EE184E025D810FF03C06C
:1013100061E084E002C061E085E096D71F5F8981CB
:10132000811778F780E0C6D79E012D5F3F4FAE0151
:101330004C5F5F4FBE016E5F7F4F81E04DD8C6DCD2
:1013400062E085E081D78A818230A0F08B8188239A
:1013500051F0419A2D9A62E085E076D741982D9818
:1013600064E085E071D72D9A419A21E040E062ED7A
:101370008AE0F1D7298181E090E0821B9109880FF2
:10138000991FEE27FF27E81BF90BE055FF4F8591CA
:1013900094910196880F991F9093090180930801F9
:1013A0001092B20083B5826083BD8091700081602D
:1013B0008093700080E07ED7809170008E7F809354
:1013C00070008A818130D9F4809104018330B9F4AE
:1013D0008B81882351F0419A2D9A62E085E034D7C1
:1013E00041982D9864E085E02FD72D9A419A21E00D
:1013F00040E062ED8AE0AFD764E085E025D72D9824
:10140000419876DA8FD761E085E01ED788E028E141
:1014100030E00FB6F894A895209360000FBE80933B
:10142000600083B7817F846083BFFFCFDF93CF935A
:1014300000D000D0CDB7DEB787E08093050180E013
:1014400039D79E012E5F3F4FAE014D5F5F4FBE010A
:101450006F5F7F4F81E0C0D739DC809164008E7F61
:101460008093640061E083E0EFD6F999FECF8CE0D1
:1014700090E092BD81BDF89A60B5F999FECF8BE0FE
:1014800090E092BD81BDF89A80B5A7D680B78860FC
:1014900080BF85E090E020E80FB6F89420936100CB
:1014A000809361000FBE5B9A0000000089B15B98D9
:1014B00083FDF9CF80B7877F80BF2D9819DA32D7A7
:1014C00028E088E190E00FB6F894A895809360003A
:1014D0000FBE2093600083B7817F846083BFFFCFFE
:1014E00085E0809305011092060180E0E3D61AD7CB
:1014F000EDDBF999FECF8BE090E092BD81BDF89ACB
:1015000080B561E06AD685E090E020E80FB6F894F7
:1015100020936100809361000FBE8091B6008062CD
:101520008093B6008091B10082608093B1001092E8
:10153000B200809170008160809370001092B400BE
:101540008091B60082FDFCCFABD683B7817F83BF8D
:1015500083B7816083BF889583B78E7F83BF5B9A93
:101560000000000089B15B9883FDEFCF80B7877FD3
:1015700080BF80B7806880BF2D98BAD9D3D628E0C5
:1015800088E190E00FB6F894A895809360000FBEB4
:101590002093600083B7817F846083BFFFCF0F9368
:1015A0001F93DF93CF9300D000D0CDB7DEB7182FB5
:1015B00087E08093050182E08093060180E07AD67F
:1015C0009E012E5F3F4FAE014D5F5F4FBE016F5FCB
:1015D0007F4F81E001D77ADB113091F4F999FECF8A
:1015E00080E090E092BD81BDF89A80B590E0880FD0
:1015F000991F80569F4FFC0125913491F90109955F
:10160000F999FECF8AE090E092BD81BDF89A00B5CD
:10161000F999FECF8BE090E092BD81BDF89A80B53C
:1016200061E0DBD585E090E020E80FB6F8942093E8
:101630006100809361000FBE8091B600806280934C
:10164000B6008091B10082608093B1001092B20028
:10165000809170008160809370001092B40080913E
:10166000B60082FDFCCF1CD6998183B7817F83BFF2
:1016700083B7816083BF889583B78E7F83BF113026
:1016800041F4809106018230A0F464E083E0DCD56F
:1016900017C0923029F480910601081750F404C055
:1016A00080910601813128F02D98419880B788609B
:1016B00080BF5B9A0000000089B15B9883FDD5CFA5
:1016C00080B7877F80BF80B7806880BF2D984198A2
:1016D000809170008E7F80937000113091F4F999A1
:1016E000FECF80E090E092BD81BDF89A80B590E099
:1016F000880F991F80569F4FFC0125913491F90165
:101700000995F6D80FD688E028E130E00FB6F894B6
:10171000A895209360000FBE8093600083B7817FFF
:10172000846083BFFFCFCF92DF92EF92FF920F933F
:101730001F93DF93CF9300D000D0CDB7DEB786E004
:101740008093050180E0B6D59E012E5F3F4FAE012C
:101750004D5F5F4FBE016F5F7F4F81E03DD6B6DAD0
:1017600085E090E020E80FB6F89420936100809324
:1017700061000FBE62E083E067D59BE0C92E90E078
:10178000D92E81E0E82EF12C8091B6008062809302
:10179000B6008091B10083608093B1001092B200D6
:1017A0001092B4008091B60082FDFCCF419A2D9A30
:1017B00021E040E062ED8AE0CED521E040E062ED3C
:1017C0008AE0C9D52D98419862E083E03DD5F9992A
:1017D000FECFD2BCC1BCF89A80B561E0FED460D522
:1017E00081E0809306018091700081608093700099
:1017F00083B7817F83BF83B7816083BF889583B7B9
:101800008E7F83BF80910601882309F04EC080B788
:10181000877F80BF80B7806880BF419A2D9A2981D9
:101820002130D9F48B819C810897B8F080917000A9
:101830008E7F8093700040E062ED8AE08CD500E0FE
:1018400010E005C061E082E0FFD40F5F1F4F8B8185
:101850009C8108171907B0F324C0C701821B9109A6
:10186000880F991FEE27FF27E81BF90BE055FF4F64
:1018700085919491880F991F880F991F01969093D5
:1018800003018093020180910201909103019093E2
:101890000901809308018091080190910901892B29
:1018A000D1F741982D9860E115C0809106018637E7
:1018B000A0F080B7877F80BF80B7806880BF8091AD
:1018C00070008E7F8093700021E040E065E080EF43
:1018D00042D56EE083E0B8D457CF5B9A0000000099
:1018E00089B15B9883FD84CF80B7877F80BF80B745
:1018F000806880BF809170008E7F80937000419AD5
:101900002D9A21E040E062ED8AE025D52D9841989E
:1019100062E083E099D4ECD705D528E088E190E037
:101920000FB6F894A895809360000FBE20936000D6
:1019300083B7817F846083BFFFCF23E045E062E30C
:1019400085E009D5089588E028E130E00FB6F894E5
:10195000A895209360000FBE8093600083B7817FBD
:10196000846083BFFFCF0F931F93F999FECF80E070
:1019700090E092BD81BDF89A80B5E82FF0E0EE0FBF
:10198000FF1FE056FF4F0591149180E093D4F801BA
:101990000995C8D461E084E057D428E088E190E05C
:1019A0000FB6F894A895809360000FBE2093600056
:1019B00083B7817F846083BFFFCF3091610087E070
:1019C00090E020E80FB6F8942093610080936100C6
:1019D0000FBE81E088B918B888B918B888B918B8A6
:1019E00088B918B888B918B888B918B888B918B8B3
:1019F00088B918B888B918B888B918B888B918B8A3
:101A000088B918B888B918B888B918B888B918B892
:101A100088B918B880E000008F5F8A35E1F781E06F
:101A200088B918B888B918B888B918B888B918B872
:101A300088B918B888B918B888B918B888B918B862
:101A400088B918B888B918B888B918B888B918B852
:101A500088B918B888B918B888B918B888B918B842
:101A60003F7080E80FB6F894809361003093610076
:101A70000FBE0895CF93DF934091610083E090E023
:101A800020E80FB6F89420936100809361000FBEA8
:101A900030E023E051E0C4EFDAE1A7E7B1E0E5E4AC
:101AA000F3E068EB7DE342C058B9822F8A95F1F7E5
:101AB00018B8822F8A95F1F700009F5F9C34A1F738
:101AC000CE010197F1F790E058B9822F8A95F1F78E
:101AD00018B8822F8A95F1F700009F5F9F30A1F719
:101AE000CD010197F1F790E058B9822F8A95F1F76F
:101AF00018B8822F8A95F1F700009F5F9031A1F707
:101B0000CF010197F1F790E058B9822F8A95F1F74C
:101B100018B8822F8A95F1F700009F5F9031A1F7E6
:101B2000CB010197F1F73F5F323011F090E0BCCF6D
:101B30004F7080E80FB6F894809361004093610085
:101B40000FBEDF91CF9108954091610081E090E058
:101B500020E80FB6F89420936100809361000FBED7
:101B600080E090E051E031E158B9232F2A95F1F758
:101B700018B8232F2A95F1F7019621E0863D9207A8
:101B800099F788EB9BE00197F1F720E030E051E115
:101B9000E1E068EE73E013C0E8B9852F8A95F1F7AC
:101BA00018B8852F8A95F1F79F5F9632A9F7CB0178
:101BB0000197F1F72F5F3F4F2730310511F090E08B
:101BC000EBCF4F7080E80FB6F8948093610040939C
:101BD00061000FBE08950F931F937091610081E023
:101BE00090E020E80FB6F8942093610080936100A4
:101BF0000FBE80E090E041E030E148B9232F2A9504
:101C0000F1F718B8232F2A95F1F7019621E08E35C8
:101C1000920799F78CEC90E10197F1F790E031E0B1
:101C200020E138B9822F8A95F1F718B8822F8A956A
:101C3000F1F79F5F9631A9F760E02FE730E84CEDB0
:101C400051E6ACE1B2E0E4E0F6E010E101E057FF7C
:101C500002C0CF0101C0CD010197F1F790E008B9B2
:101C6000812F8A95F1F718B8812F8A95F1F79F5F38
:101C70009731A9F76F5F603229F0220F331F441F9D
:101C8000551FE5CF7F7080E80FB6F8948093610010
:101C9000709361000FBE1F910F910895E091610054
:101CA00081E090E020E80FB6F894209361008093E3
:101CB00061000FBE90E031E020E138B9822F8A95B3
:101CC000F1F718B8822F8A95F1F79F5F9A35A9F737
:101CD00060E020E030EF48EB54EBAEE4B2E0F1E03E
:101CE00070E1CD010197F1F757FF0DC090E0F8B911
:101CF000872F8A95F1F718B8872F8A95F1F79F5F9C
:101D00009D32A9F70CC090E0F8B9872F8A95F1F7BA
:101D100018B8872F8A95F1F79F5F9731A9F76F5F02
:101D2000643129F0220F331F441F551FDACFEF70A3
:101D300080E80FB6F89480936100E09361000FBED5
:0A1D4000089500000895F894FFCF05
:00000001FF
